:020000040000FA
:0600000014EF33F01200C2
:0600080004EF08F01200F5
:060018000CEF08F01200DD
:0610000014EF33F01200B2
:021006001200D6
:0610080056EF0BF0120090
:06101800A0EF0BF0120036
:02101E000100CF
:0C10200060660000600000005800000046
:04102C0092808050DE
:10103000010B1200D9CFE6FFE1CFD9FFD950FD0F48
:10104000E96EFF0EDA20EA6EEE50ED100BE0FD0EB9
:10105000DB06FE0E01E2DB06500EE66E22EC33F0FC
:10106000E552ECD7E552E7CFD9FF1200D9CFE6FF22
:10107000E1CFD9FFE652F29E92908090E00EE66EAC
:10108000010EE66E1EEC32F0E552E5529290808041
:10109000280EE66EE66A1EEC32F0E552E552C6DF37
:1010A000DF6EA80EE66E010EE66E1EEC32F0E55223
:1010B000E552F28EDF50E552E552E7CFD9FF12003C
:1010C000D9CFE6FFE1CFD9FFE652F29E9290809011
:1010D000020EE66EE66A1EEC32F0E552E552A6DF3D
:1010E000050EE66EE66A1EEC32F0E552E5529EDF32
:1010F000DF6EF28EDF50E552E552E7CFD9FF1200E6
:10110000D9CFE6FFE1CFD9FFF29E92908090020EF8
:10111000E66EE66A1EEC32F0E552E552FE0EDB505A
:1011200002E092908080640EE66EE66A1EEC32F079
:10113000E552E55292908080F28EE552E7CFD9FFDA
:101140001200D9CFE6FFE1CFD9FF020EE126010E52
:10115000DB6ADF6A080EDF5C1EE2B2DF000912E024
:10116000010EDF5206E0DFCFF3FFE846FE0BF30689
:10117000FCE1146E010EDBCFE7FF1450E712010E05
:10118000E7CFDBFF780EE66EE66A1EEC32F0E55242
:10119000E552DF2ADFD7010EDB50146E020EE15C50
:1011A00002E2E16AE552E16E1450E552E7CFD9FF61
:1011B0001200D9CFE6FFE1CFD9FF020EE126DF6AA8
:1011C000080EDF5C1BE2FE0EDB50DF5206E0DFCFD5
:1011D000F3FFE8327F0BF306FCE1E76E010EE7CF89
:1011E000DBFFDB92DB94DB96DB98DB9ADB9CDB9E00
:1011F000DBCFE6FF85DFE552DF2AE2D7690EE66E38
:10120000E66A1EEC32F0E552E552020EE15C02E2C3
:10121000E16AE552E16EE552E7CFD9FF1200D9CF7E
:10122000E6FFE1CFD9FFE652FE0EDB50550814E190
:10123000550EE66EBEDFE552DF6A080EDF5C10E297
:10124000DF50EA6AF40FE96E000EEA22EF50E66E14
:10125000B0DFE552DF2AF1D7CC0EE66EAADFE55209
:10126000E552E552E7CFD9FF1200D9CFE6FFE1CF33
:10127000D9FF080EE126010EF36E020EF3CFDBFF5D
:10128000010EF36E030EF3CFDBFF040EDB6A070ED5
:10129000DB6A010EDB6A080EF36E010EDBCFF4FF92
:1012A000F350F45C0BE2010EDB50EA6AF40FE96ED6
:1012B000000EEA22EF6A010EDB2AEDD7D7DEE76ED9
:1012C000060EE7CFDBFFDB5003E10001FC5104E039
:1012D0000001FD6B000EABD0F00EE66E6ADFE5524A
:1012E000010EDB6ADF6AECDE000902E0020EDF6E4F
:1012F000780EE66EE66A1EEC32F0E552E552E0DE6C
:10130000000902E0000EDF80780EE66EE66A1EEC51
:1013100032F0E552E552030EDF5C6DE0DF5000086D
:1013200005E2DF407F0BE76E050E2BD00001FD517B
:10133000F36E030EDBCFF4FFF350F45C11E2020E08
:10134000DBCFE6FF010EDB50EA6AF40FE96E000E18
:10135000EA22EF50E552E714000806E2010E07D03A
:10136000030EDB50FD5D02E0000E01D0010EE76EC2
:10137000050EE7CFDBFFDB5006E1030EDB50E76E27
:10138000040EE7CFDBFF050EDB500BE0010EDB5058
:10139000EA6AF40FE96E000EEA22020EDB50EF1249
:1013A0000CD0020EDB1C146E010EDB50EA6AF40F47
:1013B000E96E000EEA221450EF16050EDBCFE6FFB1
:1013C0009FDEE552030EDB2A020EDB50020D020EF9
:1013D000F3CFDBFFDB5006E1010EDB2AF36E020EDA
:1013E000F3CFDBFF080EF36E010EDBCFF4FFF350FB
:1013F000F45C01E277D7410EF36E030EDBCFF4FF0E
:10140000F350F45C03E20001FD6B0FD0040EDBCF60
:10141000FDF00001FD5102E0000E01D0010EFC6F55
:10142000010EF36E070EF3CFDBFF070EDB50146ED9
:10143000080EE15C02E2E16AE552E16E1450E55209
:10144000E7CFD9FF12000001FD6BFC6B35EF09F00F
:10145000D9CFE6FFE1CFD9FF09DE550EE66EDFDE1C
:10146000E5524E0EE66EA5DEE552FE0EDBCFE6FF40
:10147000A0DEE552FD0EDBCFE6FF9BDEE5520A0E55
:10148000E66EE66A1EEC32F0E552E552EFDD550EEF
:10149000E66EC5DEE552480EE66E8BDEE5520A0EBC
:1014A000E66EE66AC7DDE552E552E552E7CFD9FFC1
:1014B0001200D9CFE6FFE1CFD9FF0E0EE126D6DD2F
:1014C000550EE66EACDEE552BE0EE66E72DEE552FD
:1014D000DF6A090EDF5C13E234DEE66ED950050FD9
:1014E000146EDACF15F0DF500F011424E96E000EF0
:1014F000DA20EA6EE552E750EF6EDF2AEAD7B6DD72
:10150000550EE66E8CDEE55292908080440EE66EBB
:1015100050DEE552050EDB50FF0808E10C0EDB50F3
:10152000100804E0F36A800EF46EB6D0010EDB6A98
:10153000020EDB6A060EDBCF14F014C015F0146A3D
:10154000010E14C0DBFF020E15C0DBFF050EDB50E1
:10155000146E156AD950010FE96EDACFEAFF145004
:10156000EE121550ED12100E0001F45D74E1D95029
:10157000010FE96EDACFEAFF010E0F0B06E0EC5225
:10158000D890ED32EF32E806FAE1010EDBCF14F02D
:10159000020EDBCF15F014C015F0146A010E14C052
:1015A000DBFF020E15C0DBFFD950010FE96EDACF69
:1015B000EAFF400EEE5E000EED5A0C0EDBCFE6FFAA
:1015C0000B0EDB50E552E75CE66ED950030FE96E77
:1015D000DACFEAFFE552E750EE6EED6A030EDBCF9D
:1015E00014F0040EDBCF15F014C015F0146A030ECE
:1015F00014C0DBFF040E15C0DBFF0C0EDB5016E041
:101600000C0EDB50146E156A030EDBCF08F0040ECF
:10161000DBCF09F014C00DF015C00EF0EEEC32F087
:10162000030E08C0DBFF040E09C0DBFF010EDBCF99
:1016300016F0020EDBCF17F0030EDB501624146EEB
:10164000040EDB501720156E030E14C0DBFF040ED2
:1016500015C0DBFF17D0010EDBCF08F0020EDBCF89
:1016600009F0030E08C0DBFF040E09C0DBFFD950F0
:10167000030FE96EDACFEAFF040ED890EE36ED36AE
:10168000E806FBE1030EDBCF14F0040EDBCF15F010
:1016900014C0F3FF15C0F4FF0E0EE15C02E2E16A34
:1016A000E552E16EE552E7CFD9FF1200DACFE4FF51
:1016B000E2CFDAFFE9CFE4FFEACFE4FFF6CFE4FFC1
:1016C000F7CFE4FFF5CFE4FFF3CFE4FFF4CFE4FF7F
:1016D000FACFE4FF00EE00F0140EE80403E3EECFCF
:1016E000E4FFFBD700EE14F0080EE80403E3EECFAE
:1016F000E4FFFBD7E6520CD9E55200EE1BF0080ED2
:10170000E80403E3E5CFEDFFFBD700EE13F0140E82
:10171000E80403E3E5CFEDFFFBD7E5CFFAFFE5CF24
:10172000F4FFE5CFF3FFE5CFF5FFE5CFF7FFE5CF1A
:10173000F6FFE5CFEAFFE5CFE9FFE5CFDAFF1100DD
:10174000D8CFE4FFE0CFE4FFE46EDACFE4FFE2CFEE
:10175000DAFFE9CFE4FFEACFE4FFF6CFE4FFF7CF0B
:10176000E4FFF5CFE4FFF3CFE4FFF4CFE4FFFACFDB
:10177000E4FF00EE00F0140EE80403E3EECFE4FF14
:10178000FBD700EE14F0080EE80403E3EECFE4FF0D
:10179000FBD7E65253D9E55200EE1BF0080EE804E1
:1017A00003E3E5CFEDFFFBD700EE13F0140EE804E2
:1017B00003E3E5CFEDFFFBD7E5CFFAFFE5CFF4FF7D
:1017C000E5CFF3FFE5CFF5FFE5CFF7FFE5CFF6FF78
:1017D000E5CFEAFFE5CFE9FFE5CFDAFFE550E5CF5A
:1017E000E0FFE5CFD8FF1000D9CFE6FFE1CFD9FF6A
:1017F000020EE12660DA5AEC2FF0200E0001B85DEF
:1018000002E05AEC2FF00001F251F31105E0A8ECD0
:1018100019F00001F26BF36B00019C519D116FE018
:101820009051911118E1A86BA96B060EA7AF02D0D9
:10183000D89003D0A65D000EA75904E2A62B000E97
:10184000A72309D0A66BA76BFEDD000904E0010EFB
:101850000001906F916B00019051911144E029DEDD
:10186000F3CFDEFFF4CFDDFFDECF14F0DDCF15F0D8
:10187000153404E314500008C90E15541AE2DECFE3
:1018800016F0DDCF17F0D890175004E6000E165C66
:101890007D0E17580EE20001A86BA96B92519311AF
:1018A00005E0DECF94F0DDCF95F01DD09269936B0B
:1018B0001AD00001A82B000EA923A93514E2A851C3
:1018C0000408000EA9550FE2946B800E956F906B83
:1018D000916B926B936B030E9E1905E19F5103E18F
:1018E000020E9E6F9F6B9C6B9D6B9E519F1107E03C
:1018F000050E7C1901E17D5102E0BCEC1AF039ECD7
:101900001CF00001B25101E178D7A5EC24F075D7A5
:101910000001B551B61102E1000E08D0B5C0E9FFD3
:10192000B6C0EAFFEF50800B01E0010E000901E0B4
:1019300083D0200E0001B85D01E07ED0040130515B
:10194000730A01E177D0010A72E0020A6DE0110A20
:1019500068E0010A63E0310A5EE0100A59E07A0AA1
:1019600054E0010A4FE0030A4AE0010A45E00F0A89
:1019700040E0010A3BE0030A36E0010A31E0070AD1
:101980002CE0010A27E0030A22E0010A1DE0190AFF
:1019900018E0010A13E0090A0EE0010A09E0310A21
:1019A00004E0010A49E1DCDB47D04EEC11F044D001
:1019B0009BEC11F041D0F2EC11F03ED042EC12F071
:1019C0003BD088EC12F038D0CEEC12F035D016ECCB
:1019D00013F032D052EC13F02FD0A8EC13F02CD02F
:1019E000E6EC13F029D04BEC14F026D087EC14F081
:1019F00023D0EDEC14F020D030EC15F01DD0B0EC7D
:101A000015F01AD0F5EC15F017D06EEC16F014D0D6
:101A1000ACEC16F011D0FAEC16F00ED038EC17F052
:101A20000BD080EC17F008D0BCEC17F005D088EC98
:101A300018F002D062EC19F0F5EF26F0D9CFE6FFEE
:101A4000E1CFD9FF020EE1269E90CD90F00ECF6E31
:101A5000CD800001D890635104E6FF0E625D010E57
:101A6000635904E2622B000E63231CD0626B636B2C
:101A7000050E7C1903E17D5101E18A70010E9E196A
:101A800001E19F5105E0020E9E190CE19F510AE110
:101A90006C516D1107E189788950100B02E0898A39
:101AA00001D0899AD8909B5104E6880E9A5D130E56
:101AB0009B5904E29A2B000E9B2305D09A6B9B6BDB
:101AC000010E9C6F9D6B8150DE6EDD6ADECF14F0DF
:101AD000DDCF15F0141E151E14C0DEFF15C0DDFF8E
:101AE000DECF14F0DDCF15F0040ED890153214328D
:101AF000E804FBE1030E00011414866F876B070EE8
:101B00008E1901E18F5101E18ED0060E8E1901E18F
:101B10008F5101E176D0050E8E1901E18F5163E0FE
:101B2000030E8E1901E18F514AE0020E8E1901E178
:101B30008F5133E0010E8E1901E18F5120E08E515B
:101B400001E18F510CE0040E8E1901E082D08F511B
:101B500001E07FD08651871101E07ED06AD0020E6D
:101B6000861902E1875125E0010E861902E18751AD
:101B700054E0030E861970E187516EE168D0030EC0
:101B8000861902E1875127E08651871152E0010E44
:101B9000861962E1875160E15AD0010E861904E18D
:101BA000875102E1030E56D0020E861904E18751D7
:101BB00002E1010E4FD0865187114EE13AD0865195
:101BC000871104E18C2B000E8D2333D0030E861970
:101BD00004E1875102E1020E3DD0020E86193CE17C
:101BE00087513AE134D0030E861902E1875128E08B
:101BF000865187111EE0020E86192EE187512CE1D5
:101C000026D0020E861904E1875102E1070E22D088
:101C1000010E861904E1875102E1050E1BD08651A1
:101C200087111AE106D08651871105E18A2B000E33
:101C30008B238E6B10D0030E861904E1875102E1CD
:101C4000060E08D0010E861907E1875105E1040E42
:101C500001D0040E8E6F8F6B030E7C1922E17D5133
:101C600020E18D518B19E8AE02D08B3504D08A511A
:101C70008C5D8B518D5905E2010E8A6F8B6B8C6BDD
:101C80008D6B8B518D19E8AE02D08D3504D08C51FF
:101C90008A5D8D518B5905E28A6B8B6B010E8C6FBF
:101CA0008D6B020EE15C02E2E16AE552E16EE55203
:101CB000E7CFD9FF1200D9CFE6FFE1CFD9FFE65237
:101CC0000F0EC112F19ED08E928218D869EC26F0C8
:101CD000CD92CD96CD88CD9ACD9CCD90F00ECF6E85
:101CE000CE6ACD809F909D80F28C8150DF6EF29005
:101CF000F28EE552E552E7CFD9FF1200D9CFE6FFC9
:101D0000E1CFD9FF020EE126FC0E8A129316C70E10
:101D1000891292168998899A8A908A92300E931223
:101D20009284B80E8B1694161F0EE66E96EC24F075
:101D3000E552A50801E0FED00B0EE66E96EC24F00D
:101D4000E552146E156E146A000E1416FF0E151669
:101D500014C0E6FF15C0E6FF0A0EE66E96EC24F00E
:101D6000E552E552E7CF15F0E552E7CF14F0000158
:101D70001410E66F15C0E7F00C0EE66E96EC24F03A
:101D8000E5520F0B0001E86FE96B0E0EE66E96EC64
:101D900024F0E552146E156E146A000E1416FF0E30
:101DA000151614C0E6FF15C0E6FF0D0EE66E96ECA4
:101DB00024F0E552E552E7CF15F0E552E7CF14F0F5
:101DC00000011410EE6F15C0EFF00F0EE66E96ECEA
:101DD00024F0E5520F0B0001F06FF16BE66A96EC10
:101DE00024F0E55200016E6F6F6B010EE66E96EC0B
:101DF00024F0E5520001706F716B020EE66E96ECF6
:101E000024F0E5520001766F776B030EE66E96ECD8
:101E100024F0E5520001786F796B040EE66E96ECC3
:101E200024F0E5520001686F696B050EE66E96ECD2
:101E300024F0E552DE6EDD6A000EDFCF08F0010E01
:101E4000DBCF09F075EC2FF007C014F008C015F0D7
:101E500009C016F00AC017F0CD0E0C6ECC0E0D6E38
:101E60000E6E410E0F6E88EC2FF056EC30F008C06D
:101E7000A2F009C0A3F0070EE66E96EC24F0E5523E
:101E8000146E156E146A14C0E6FFE66E060EE66E5A
:101E900096EC24F0E552E552E7CF15F0E552E7CF96
:101EA00014F000011410A46F15C0A5F01E0EE66E0C
:101EB00096EC24F0E5525A0839E1100EE66E96ECE5
:101EC00024F0E5520001EA6FEB6B110EE66E96EC22
:101ED00024F0E552146E156E146A14500001EA13D2
:101EE0001550EB13120EE66E96EC24F0E55200014D
:101EF000EC6FED6B130EE66E96EC24F0E5520001EC
:101F0000966F976B140EE66E96EC24F0E552146E05
:101F1000156E146A1450000196131550971396C04D
:101F200098F097C099F0020E9E6F02D000019E6B50
:101F30009F6BC3D000016E6B6F6B6EC0E6FFE66AED
:101F40006BEC24F0E552E5520001706B716B70C0D0
:101F5000E6FF010EE66E6BEC24F0E552E552280E2A
:101F60000001766F776BE66E020EE66E6BEC24F086
:101F7000E552E552010E0001786F796BE66E030EB3
:101F8000E66E6BEC24F0E552E5520001686B696B7C
:101F900068C0E6FF040EE66E6BEC24F0E552E552F5
:101FA000050EDE6EDD6A000EDFCF08F0010EDBCF1E
:101FB00009F075EC2FF007C014F008C015F009C047
:101FC00016F00AC017F0CD0E0C6ECC0E0D6E0E6E14
:101FD000410E0F6E88EC2FF056EC30F008C0A2F0E6
:101FE00009C0A3F0DFCFE6FF050EE66E6BEC24F030
:101FF000E552E5520001A46B050EA56FE66A060ED8
:10200000E66E6BEC24F0E552E552050EE66E070E27
:10201000E66E6BEC24F0E552E5520001646B656BF3
:10202000E66A080EE66E6BEC24F0E552E55200011C
:10203000E66BE76BE86BE96BE66A0A0EE66E6BEC43
:1020400024F0E552E552E66A0B0EE66E6BEC24F0E6
:10205000E552E552E66A0C0EE66E6BEC24F0E552B2
:10206000E5520001E66BE76BE86BE96BA00EE66EEC
:102070000D0EE66E6BEC24F0E552E552860EE66E30
:102080000E0EE66E6BEC24F0E552E552010EE66EA4
:102090000F0EE66E6BEC24F0E552E552E66A1E0E7A
:1020A000E66E6BEC24F0E552E552A50EE66E1F0ECF
:1020B000E66E6BEC24F0E552E5522AD80001B56BD0
:1020C000B66BB36BB46B010EB26F040E8E6F8F6B79
:1020D000030E7C6F7D6B7A697B698A908A8200012E
:1020E000F26BF36B00019A6B9B6BA66BA76BA86BF3
:1020F000A96B946B800E956F926B936B020EE15CF3
:1021000002E2E16AE552E16EE552E7CFD9FF120043
:10211000080EE66E96EC24F0E5520001646F030EA3
:102120006415646F656BB80E8B169416705171113F
:1021300016E16451651101E18B8C010E641903E114
:10214000655101E18B84020E641903E1655101E1DF
:102150008B80030E641903E1655101E18B8212004B
:10216000D9CFE6FFE1CFD9FF020EE12604013151BC
:10217000DE6EDD6A0001B351B41102E1000E08D039
:10218000B3C0E9FFB4C0EAFFEF50800B01E0010EDD
:10219000000901E079D00401100E336FDFCF35F470
:1021A0000001F251F31112E1DECF14F0DDCF15F092
:1021B000060E145C000E15581CE3D9CFE9FFDACFE8
:1021C000EAFFFF0EEE1801E1ED5013E0F251F311BA
:1021D00033E0D9CFE9FFDACFEAFFEE50ED1009E0A6
:1021E000D9CFE9FFDACFEAFFFF0EEE1825E1ED5077
:1021F00023E10401346BD9CFE9FFDACFEAFFFF0E08
:10220000EE1811E1ED500FE10001010E6C1901E132
:102210006D5105E0020E6C1911E16D510FE1010ED7
:10222000746F756B0BD0DECF6AF0DDCF6BF0010EF3
:102230000001F26FF36B02D004013469040EE66E04
:10224000330EE66E040EE66E010EE66EE66E84EC6C
:102250002EF0146E050EE15E1450F3CFB3F0F4CF00
:10226000B4F0400EE66E300EE66E040EE66EE66AE0
:10227000010EE66E84EC2EF0146E050EE15E145035
:10228000F3CFB5F0F4CFB6F0020EE15C02E2E16A02
:10229000E552E16EE552E7CFD9FF12000001B351DC
:1022A000B41102E1000E08D0B3C0E9FFB4C0EAFFE8
:1022B000EF50800B01E0010E00093CE10401110E1A
:1022C000336F0001050E7C1906E17D5104E1040124
:1022D000050E346F09D00001F251F31103E16CC017
:1022E00034F402D06AC034F4040EE66E330EE66EA7
:1022F000040EE66E010EE66EE66E84EC2EF0146EB1
:10230000050EE15E1450F3CFB3F0F4CFB4F0400EFD
:10231000E66E300EE66E040EE66EE66A010EE66EBE
:1023200084EC2EF0146E050EE15E1450F3CFB5F080
:10233000F4CFB6F012000001F251F31110E132C4F3
:1023400014F014C015F0146A000E1416FF0E1516C2
:102350000401315100011410B06F15C0B1F000013B
:10236000B351B41102E1000E08D0B3C0E9FFB4C00C
:10237000EAFFEF50800B01E0010E000932E1040199
:10238000200E336F0001B0510401346FB1C014F05E
:10239000156A1450356F040EE66E330EE66E040EA9
:1023A000E66E010EE66EE66E84EC2EF0146E050EFF
:1023B000E15E1450F3CFB3F0F4CFB4F0400EE66E0C
:1023C000300EE66E040EE66EE66A010EE66E84ECF2
:1023D0002EF0146E050EE15E1450F3CFB5F0F4CF7D
:1023E000B6F012000001B351B41102E1000E08D0A2
:1023F000B3C0E9FFB4C0EAFFEF50800B01E0010E6B
:1024000000093FE10401210E336F0001AA51AB1115
:1024100006E0AC510401346FADC014F006D00001E9
:10242000E6510401346FE7C014F0156A1450356F9B
:102430000001AA6BAB6B040EE66E330EE66E040E63
:10244000E66E010EE66EE66E84EC2EF0146E050E5E
:10245000E15E1450F3CFB3F0F4CFB4F0400EE66E6B
:10246000300EE66E040EE66EE66A010EE66E84EC51
:102470002EF0146E050EE15E1450F3CFB5F0F4CFDC
:10248000B6F012000001F251F31106E10F0E040143
:1024900031150001AE6FAF6B0001B351B41102E111
:1024A000000E08D0B3C0E9FFB4C0EAFFEF50800BC4
:1024B00001E0010E00092BE10401280E336FAEC0CC
:1024C00034F4040EE66E330EE66E040EE66E010E74
:1024D000E66EE66E84EC2EF0146E050EE15E14508E
:1024E000F3CFB3F0F4CFB4F0400EE66E300EE66EEC
:1024F000040EE66EE66A010EE66E84EC2EF0146EB3
:10250000050EE15E1450F3CFB5F0F4CFB6F0120033
:102510000001B351B41102E1000E08D0B3C0E9FFCD
:10252000B4C0EAFFEF50800B01E0010E000935E175
:102530000401290E336FE6C0ACF0E7C0ADF0000136
:10254000AA69AB6B0F0E0001E8150401346F040E8D
:10255000E66E330EE66E040EE66E010EE66EE66E75
:1025600084EC2EF0146E050EE15E1450F3CFB3F040
:10257000F4CFB4F0400EE66E300EE66E040EE66E5A
:10258000E66A010EE66E84EC2EF0146E050EE15E36
:102590001450F3CFB5F0F4CFB6F01200040131516E
:1025A0000001766F776BE66E020EE66E6BEC24F040
:1025B000E552E5520001B351B41102E1000E08D01A
:1025C000B3C0E9FFB4C0EAFFEF50800B01E0010E99
:1025D00000092BE10401300E336F76C034F4040E91
:1025E000E66E330EE66E040EE66E010EE66EE66EE5
:1025F00084EC2EF0146E050EE15E1450F3CFB3F0B0
:10260000F4CFB4F0400EE66E300EE66E040EE66EC9
:10261000E66A010EE66E84EC2EF0146E050EE15EA5
:102620001450F3CFB5F0F4CFB6F012000001B3515F
:10263000B41102E1000E08D0B3C0E9FFB4C0EAFF54
:10264000EF50800B01E0010E00092BE10401310E77
:10265000336F76C034F4040EE66E330EE66E040E6D
:10266000E66E010EE66EE66E84EC2EF0146E050E3C
:10267000E15E1450F3CFB3F0F4CFB4F0400EE66E49
:10268000300EE66E040EE66EE66A010EE66E84EC2F
:102690002EF0146E050EE15E1450F3CFB5F0F4CFBA
:1026A000B6F01200040131510001786F796BE66ECB
:1026B000030EE66E6BEC24F0E552E5520401325154
:1026C0000001686F696BE66E040EE66E6BEC24F039
:1026D000E552E5520001B351B41102E1000E08D0F9
:1026E000B3C0E9FFB4C0EAFFEF50800B01E0010E78
:1026F00000092DE10401320E336F78C034F468C054
:1027000035F4040EE66E330EE66E040EE66E010E30
:10271000E66EE66E84EC2EF0146E050EE15E14504B
:10272000F3CFB3F0F4CFB4F0400EE66E300EE66EA9
:10273000040EE66EE66A010EE66E84EC2EF0146E70
:10274000050EE15E1450F3CFB5F0F4CFB6F01200F1
:102750000001B351B41102E1000E08D0B3C0E9FF8B
:10276000B4C0EAFFEF50800B01E0010E00092DE13B
:102770000401330E336F78C034F468C035F4040EAE
:10278000E66E330EE66E040EE66E010EE66EE66E43
:1027900084EC2EF0146E050EE15E1450F3CFB3F00E
:1027A000F4CFB4F0400EE66E300EE66E040EE66E28
:1027B000E66A010EE66E84EC2EF0146E050EE15E04
:1027C0001450F3CFB5F0F4CFB6F01200040131513C
:1027D0000001A06FA16BE66E050EE66E6BEC24F0B7
:1027E000E552E552A0C008F0A1C009F075EC2FF049
:1027F00007C014F008C015F009C016F00AC017F0A1
:10280000CD0E0C6ECC0E0D6E0E6E410E0F6E88EC62
:102810002FF056EC30F008C0A2F009C0A3F0000180
:10282000B351B41102E1000E08D0B3C0E9FFB4C047
:10283000EAFFEF50800B01E0010E00092BE10401DB
:10284000340E336FA0C034F4040EE66E330EE66E21
:10285000040EE66E010EE66EE66E84EC2EF0146E4B
:10286000050EE15E1450F3CFB3F0F4CFB4F0400E98
:10287000E66E300EE66E040EE66EE66A010EE66E59
:1028800084EC2EF0146E050EE15E1450F3CFB5F01B
:10289000F4CFB6F012000001B351B41102E1000E02
:1028A00008D0B3C0E9FFB4C0EAFFEF50800B01E0ED
:1028B000010E00092BE10401350E336FA0C034F482
:1028C000040EE66E330EE66E040EE66E010EE66E44
:1028D000E66E84EC2EF0146E050EE15E1450F3CF1C
:1028E000B3F0F4CFB4F0400EE66E300EE66E040E98
:1028F000E66EE66A010EE66E84EC2EF0146E050EAE
:10290000E15E1450F3CFB5F0F4CFB6F0120032C44C
:1029100014F014C015F0146A000E1416FF0E1516EC
:102920000401315100011410A46F15C0A5F0E85046
:10293000E66E060EE66E6BEC24F0E552E552A5C09D
:1029400014F0156A1450E66E070EE66E6BEC24F078
:10295000E552E5520001B351B41102E1000E08D076
:10296000B3C0E9FFB4C0EAFFEF50800B01E0010EF5
:10297000000932E10401360E336F0001A451040155
:10298000346FA5C014F0156A1450356F040EE66E4E
:10299000330EE66E040EE66E010EE66EE66E84EC15
:1029A0002EF0146E050EE15E1450F3CFB3F0F4CFA9
:1029B000B4F0400EE66E300EE66E040EE66EE66A89
:1029C000010EE66E84EC2EF0146E050EE15E1450DE
:1029D000F3CFB5F0F4CFB6F012000001B351B4114B
:1029E00002E1000E08D0B3C0E9FFB4C0EAFFEF5027
:1029F000800B01E0010E000932E10401370E336F54
:102A00000001A4510401346FA5C014F0156A1450DC
:102A1000356F040EE66E330EE66E040EE66E010EA2
:102A2000E66EE66E84EC2EF0146E050EE15E145038
:102A3000F3CFB3F0F4CFB4F0400EE66E300EE66E96
:102A4000040EE66EE66A010EE66E84EC2EF0146E5D
:102A5000050EE15E1450F3CFB5F0F4CFB6F01200DE
:102A6000040131512BE000019E519F112AE1905148
:102A7000911117E0945102E1800E951912E0E6C021
:102A8000EAF0E7C0EBF0E8C0ECF0E9C0EDF094C08C
:102A900096F095C097F094C098F095C099F0030E09
:102AA0000BD00001EA6BEB6BEC6BED6B0001966BEE
:102AB000976B986B996B010E9E6F02D000019E6B15
:102AC0009F6BB351B41102E1000E08D0B3C0E9FF0F
:102AD000B4C0EAFFEF50800B01E0010E000934E1C1
:102AE0000401380E336F0001030E9E1905E19F515A
:102AF00003E10401346902D00401346B040EE66E74
:102B0000330EE66E040EE66E010EE66EE66E84ECA3
:102B10002EF0146E050EE15E1450F3CFB3F0F4CF37
:102B2000B4F0400EE66E300EE66E040EE66EE66A17
:102B3000010EE66E84EC2EF0146E050EE15E14506C
:102B4000F3CFB5F0F4CFB6F00001030E9E1905E106
:102B50009F5103E18988898A12008998899A120015
:102B60000001B351B41102E1000E08D0B3C0E9FF77
:102B7000B4C0EAFFEF50800B01E0010E000934E120
:102B80000401390E336F0001030E9E1905E19F51B8
:102B900003E10401346902D00401346B040EE66ED3
:102BA000330EE66E040EE66E010EE66EE66E84EC03
:102BB0002EF0146E050EE15E1450F3CFB3F0F4CF97
:102BC000B4F0400EE66E300EE66E040EE66EE66A77
:102BD000010EE66E84EC2EF0146E050EE15E1450CC
:102BE000F3CFB5F0F4CFB6F012000401315122E179
:102BF0000001706B716B050E7C1901E17D5128E0BD
:102C0000B80E8B1694166451651101E18B8C010E80
:102C1000641903E1655101E18B84020E641903E13B
:102C2000655101E18B80030E641912E1655110E1D9
:102C30008B820ED000017069716B010E6C1901E17D
:102C40006D5106E0020E6C1901E16D5101E08B6AD5
:102C50007051E66E010EE66E6BEC24F0E552E55223
:102C60000001B351B41102E1000E08D0B3C0E9FF76
:102C7000B4C0EAFFEF50800B01E0010E00092DE126
:102C800004013A0E336F000170510401346F040ED9
:102C9000E66E330EE66E040EE66E010EE66EE66E2E
:102CA00084EC2EF0146E050EE15E1450F3CFB3F0F9
:102CB000F4CFB4F0400EE66E300EE66E040EE66E13
:102CC000E66A010EE66E84EC2EF0146E050EE15EEF
:102CD0001450F3CFB5F0F4CFB6F012000001B351A9
:102CE000B41102E1000E08D0B3C0E9FFB4C0EAFF9E
:102CF000EF50800B01E0010E00092DE104013B0EB5
:102D0000336F000170510401346F040EE66E330E10
:102D1000E66E040EE66E010EE66EE66E84EC2EF0B4
:102D2000146E050EE15E1450F3CFB3F0F4CFB4F09F
:102D3000400EE66E300EE66E040EE66EE66A010E9A
:102D4000E66E84EC2EF0146E050EE15E1450F3CFA7
:102D5000B5F0F4CFB6F012000001B351B41102E1A6
:102D6000000E08D0B3C0E9FFB4C0EAFFEF50800BFB
:102D700001E0010E00093DE10401410E336F000145
:102D800091350DE290510008000E915508E29451E2
:102D90000401346F95C014F0156A145003D0040177
:102DA000346B800E356F040EE66E330EE66E040E45
:102DB000E66E010EE66EE66E84EC2EF0146E050EE5
:102DC000E15E1450F3CFB3F0F4CFB4F0400EE66EF2
:102DD000300EE66E040EE66EE66A010EE66E84ECD8
:102DE0002EF0146E050EE15E1450F3CFB5F0F4CF63
:102DF000B6F012000001B351B41102E1000E08D088
:102E0000B3C0E9FFB4C0EAFFEF50800B01E0010E50
:102E100000092DE10401510E336F020E346F050ECF
:102E2000356F040EE66E330EE66E040EE66E010E8E
:102E3000E66EE66E84EC2EF0146E050EE15E145024
:102E4000F3CFB3F0F4CFB4F0400EE66E300EE66E82
:102E5000040EE66EE66A010EE66E84EC2EF0146E49
:102E6000050EE15E1450F3CFB5F0F4CFB6F01200CA
:102E7000010E0401311500016E6F6F6BE66EE66A9C
:102E80006BEC24F0E552E5520001B351B41102E1BC
:102E9000000E08D0B3C0E9FFB4C0EAFFEF50800BCA
:102EA00001E0010E00092BE10401600E336F6EC0DA
:102EB00034F4040EE66E330EE66E040EE66E010E7A
:102EC000E66EE66E84EC2EF0146E050EE15E145094
:102ED000F3CFB3F0F4CFB4F0400EE66E300EE66EF2
:102EE000040EE66EE66A010EE66E84EC2EF0146EB9
:102EF000050EE15E1450F3CFB5F0F4CFB6F012003A
:102F00000001B351B41102E1000E08D0B3C0E9FFD3
:102F1000B4C0EAFFEF50800B01E0010E00092BE185
:102F20000401610E336F6EC034F4040EE66E330E8E
:102F3000E66E040EE66E010EE66EE66E84EC2EF092
:102F4000146E050EE15E1450F3CFB3F0F4CFB4F07D
:102F5000400EE66E300EE66E040EE66EE66A010E78
:102F6000E66E84EC2EF0146E050EE15E1450F3CF85
:102F7000B5F0F4CFB6F01200D9CFE6FFE1CFD9FF1C
:102F8000020EE126DE68DD6AA50E0401315D01E076
:102F90007AD000016C516D1176E10001E651E66EC8
:102FA0000A0EE66E6BEC24F0E552E552E7C014F031
:102FB000156A1450E66E0B0EE66E6BEC24F0E552CB
:102FC000E5520F0E0001E815E66E0C0EE66E6BEC96
:102FD00024F0E552E5520001030E9E194AE19F518B
:102FE00048E10001EA51E66E100EE66E6BEC24F04B
:102FF000E552E552EBC014F0156A1450E66E110E5E
:10300000E66E6BEC24F0E552E552ECC0E6FF120EE2
:10301000E66E6BEC24F0E552E55200019651E66E47
:10302000130EE66E6BEC24F0E552E55297C014F0F7
:10303000156A1450E66E140EE66E6BEC24F0E55241
:10304000E5525A0EE66E1E0EE66E6BEC24F0E5526B
:10305000E55264C0E6FF080EE66E6BEC24F0E55224
:10306000E5528B6A8A908A92050E00017C6F7D6B17
:1030700007D0E66A1E0EE66E6BEC24F0E552E552D0
:10308000A50EDE6EDD6A0001B351B41102E1000E3F
:1030900008D0B3C0E9FFB4C0EAFFEF50800B01E0F5
:1030A000010E00092BE10401700E336FDFCF34F401
:1030B000040EE66E330EE66E040EE66E010EE66E4C
:1030C000E66E84EC2EF0146E050EE15E1450F3CF24
:1030D000B3F0F4CFB4F0400EE66E300EE66E040EA0
:1030E000E66EE66A010EE66E84EC2EF0146E050EB6
:1030F000E15E1450F3CFB5F0F4CFB6F0020EE15C10
:1031000002E2E16AE552E16EE552E7CFD9FF120033
:10311000D9CFE6FFE1CFD9FF020EE126A50E0401CB
:10312000315D72E100016C516D116EE10001E651FB
:10313000E66E0A0EE66E6BEC24F0E552E552E7C04F
:1031400014F0156A1450E66E0B0EE66E6BEC24F06C
:10315000E552E5520F0E0001E815E66E0C0EE66E24
:103160006BEC24F0E552E55264C0E6FF080EE66E13
:103170006BEC24F0E552E5528B6A8A908A92050E38
:1031800000017C6F7D6B030E9E1935E19F5133E189
:103190000001EA51E66E100EE66E6BEC24F0E5528B
:1031A000E552EBC014F0156A1450E66E110EE66E8F
:1031B0006BEC24F0E552E552ECC0E6FF120EE66E31
:1031C0006BEC24F0E552E55200019651E66E130EC9
:1031D000E66E6BEC24F0E552E55297C014F0156AE8
:1031E0001450E66E140EE66E6BEC24F0E552E552D8
:1031F0005A0EE66E01D0E66A1E0EE66E6BEC24F007
:10320000E552E552A50E15D05A0E0401315D13E1C9
:103210000001050E7C190FE17D510DE188EC10F0E5
:1032200000017C6B7D6B010E7A6F7B6B8A908A92BA
:103230005A0EDE6E01D0DE68DD6A0001B351B411B2
:1032400002E1000E08D0B3C0E9FFB4C0EAFFEF50BE
:10325000800B01E0010E00092BE10401720E336FB7
:10326000DFCF34F4040EE66E330EE66E040EE66E27
:10327000010EE66EE66E84EC2EF0146E050EE15E35
:103280001450F3CFB3F0F4CFB4F0400EE66E300E2E
:10329000E66E040EE66EE66A010EE66E84EC2EF033
:1032A000146E050EE15E1450F3CFB5F0F4CFB6F016
:1032B000020EE15C02E2E16AE552E16EE552E7CF1F
:1032C000D9FF12000001B351B41102E1000E08D081
:1032D000B3C0E9FFB4C0EAFFEF50800B01E0010E7C
:1032E000000935E10401730E336F0001050E7C19EE
:1032F00005E17D5103E10401A50E02D004015A0E3F
:10330000346F040EE66E330EE66E040EE66E010EAA
:10331000E66EE66E84EC2EF0146E050EE15E14503F
:10332000F3CFB3F0F4CFB4F0400EE66E300EE66E9D
:10333000040EE66EE66A010EE66E84EC2EF0146E64
:10334000050EE15E1450F3CFB5F0F4CFB6F01200E5
:10335000D9CFE6FFE1CFD9FF080EE126B0C0DEFFEE
:10336000B1C0DDFF020EAEC0DBFF030EAFC0DBFF5E
:10337000050E00016A1901E16B5101E1DDD0040E77
:103380006A1901E16B5101E1B6D0030E6A1901E13E
:103390006B5135E0020E6A1901E16B5122E0010E1A
:1033A0006A1901E16B5105E06A5101E0D0D06B511F
:1033B000CED0050E7C1901E17D5101E1C8D089888C
:1033C000899A000EE66EE66AD9CFE9FFDACFEAFF06
:1033D000EECFE6FFEECFE6FFEECFE6FFEFCFE6FF64
:1033E00081D0050E7C1901E17D5101E1B0D08998B1
:1033F000898A000EE66EE66AD9CFE9FF38D0050E5D
:103400007C1901E17D5101E1A2D0D9CFE9FFDACFEA
:10341000EAFFEE500001E65DEE50E759EE50E85944
:10342000EE50E95930E2D9CFE9FFDACFEAFFE651B1
:10343000EE5C146EE751EE58156EE851EE58166EBC
:10344000E951EE58176E040E14C0DBFF050E15C0CF
:10345000DBFF060E16C0DBFF070E17C0DBFF8998E7
:10346000898A000EE66EE66AD950040FE96EDACF5B
:10347000EAFFEECFE6FFEECFE6FFEECFE6FFEFCFBF
:10348000E6FF010E2FD0D9CFE9FFDACFEAFFEE50E9
:10349000E65D146EEE50E759156EEE50E859166E63
:1034A000EE50E959176E040E14C0DBFF050E15C06F
:1034B000DBFF060E16C0DBFF070E17C0DBFF898897
:1034C000899A000EE66EE66AD950040FE96EDACFEB
:1034D000EAFFEECFE6FFEECFE6FFEECFE6FFEFCF5F
:1034E000E6FF000EE66EE66A8DEC1EF0146E080E26
:1034F000E15E14502CD0DFCFE6F0010EDBCFE7F019
:10350000020EDBCFE8F0030EDBCFE9F0020E9E19CE
:1035100001E19F5105E0030E9E1919E19F5117E14A
:10352000DFCFEAF0010EDBCFEBF0020EDBCFECF0E9
:10353000030EDBCFEDF00BD0DFCFEEF0010EDBCFD3
:10354000EFF0020EDBCFF0F0030EDBCFF1F0000165
:10355000030E9E1905E19F5103E18988898A02D0F3
:103560008998899A080EE15C02E2E16AE552E16E0F
:10357000E552E7CFD9FF1200D9CFE6FFE1CFD9FF5F
:103580000A0EE12600019051911101E140D1030E94
:103590009E1901E03CD19F5101E039D19851945DD1
:1035A000146E9551995514C0DEFFDD6EDECF14F018
:1035B000DDCF15F00001800E15140CE008680968D5
:1035C000DECF0DF0DDCF0EF029EC30F006C0DEFFCF
:1035D00007C0DDFFDECF14F0DDCF15F00001A351F1
:1035E0001518E8AE02D0153404D01450A25D155061
:1035F000A35901E334D19651945D146E95519755BA
:1036000014C0DEFFDD6EA4C018F0A5C019F01A6A60
:103610001B6A19AE02D01A681B68DECF14F0DDCF2A
:1036200015F0166A176A15AE02D01668176814C02E
:1036300006F015C007F016C008F017C009F018C052
:103640000BF019C00CF01AC00DF01BC00EF061ECAD
:1036500032F002C006F003C007F004C008F005C055
:1036600009F0000E066C071E0722081E0822091E1C
:1036700009220B6A0C6A010E0D6E0E6AF5EC2FF032
:10368000060E06C0DBFF070E07C0DBFF080E08C0F2
:10369000DBFF090E09C0DBFFD950060FE96EDACF58
:1036A000EAFF0001EA51EE24146EEB51EE20156E94
:1036B000EC51EE20166EED51EE20176E020E14C086
:1036C000DBFF030E15C0DBFF040E16C0DBFF050E8B
:1036D00017C0DBFFD950020FE96EDACFEAFFE651DF
:1036E000EE5C146EE751EE58156EE851EE58166E0A
:1036F000E951EE58176E060E14C0DBFF070E15C019
:10370000DBFF080E16C0DBFF090E17C0DBFF060E3D
:10371000DBCF14F0070EDBCF15F0080EDBCF16F071
:10372000090EDBCF17F0145015101610171001E119
:1037300096D094C098F095C099F0D950060FE96ED4
:10374000DACFEAFFD890030EEB50000A08E6000E2D
:10375000EE5C000EEE58000EEE58000EEE5837E20A
:10376000060EDBCF06F0070EDBCF07F0080EDBCF2F
:1037700008F0090EDBCF09F00B680C680D680E68C5
:1037800061EC32F0060E02C0DBFF070E03C0DBFF68
:10379000080E04C0DBFF090E05C0DBFF8988899A8B
:1037A000320EE66ED7EC32F0E552020EE66EE66AB5
:1037B000D950060FE96EDACFEAFFEECFE6FFEECF83
:1037C000E6FFEECFE6FFEFCFE6FF000E18D08998B8
:1037D000898A320EE66ED7EC32F0E552020EE66EC2
:1037E000E66AD950060FE96EDACFEAFFEECFE6FFC0
:1037F000EECFE6FFEECFE6FFEFCFE6FF010EE66E7F
:10380000E66A8BDA146E080EE15E145026D09051F1
:10381000911125E0945102E1800E951920E0010EEE
:103820009E1913E19F5111E1E6C0EAF0E7C0EBF009
:10383000E8C0ECF0E9C0EDF094C096F095C097F0C8
:1038400094C098F095C099F005D0020E9E1907E13A
:103850009F5105E1030E9E6F9F6B8988898A0A0E2E
:10386000E15C02E2E16AE552E16EE552E7CFD9FFA1
:103870001200D9CFE6FFE1CFD9FF060EE1267AC0CC
:1038800014F07BC015F0166A176A15AE02D01668E0
:103890001768020E14C0DBFF030E15C0DBFF040E19
:1038A00016C0DBFF050E17C0DBFF00018D518B1921
:1038B000E8AE02D08B3504D08A518C5D8B518D5986
:1038C00008E28C518A5D8A6F8D518B598B6F8C6B9E
:1038D0008D6B8B518D19E8AE02D08D3504D08C5193
:1038E0008A5D8D518B5908E28A518C5D8C6F8B51AA
:1038F0008D598D6F8A6B8B6B040E8014040831E137
:10390000050E7C1901E17D512CE08A518B1129E0D3
:103910008A07000E8B5B8988899A320EE66ED7EC97
:1039200032F0E552010EE66EE66AD950020FE96EFA
:10393000DACFEAFFEECFE6FFEECFE6FFEECFE6FF0F
:10394000EFCFE6FF000EE66EE66AE7D9146E080ECA
:10395000E15E14500001030E9E193AE19F5135E0DB
:1039600037D0040E8014040835E1050E7C1901E1FE
:103970007D5130E08C518D112DE08C07000E8D5B58
:103980008998898A320EE66ED7EC32F0E552010E44
:10399000E66EE66AD950020FE96EDACFEAFFEECFA3
:1039A000E6FFEECFE6FFEECFE6FFEFCFE6FF010E3C
:1039B000E66EE66AB2D9146E080EE15E145000019C
:1039C000030E9E1905E19F5103E18988898A02D07F
:1039D0008998899A80B497D1DE6ADD6A040E8014D2
:1039E00016E1DECF14F0DDCF15F0D890155004E6C7
:1039F000280E145C000E15580AE2190EE66ED7EC7C
:103A000032F0E552DF2A010EE9E3DB2AE7D7DECF09
:103A100014F0DDCF15F0D890155004E6020E145CBA
:103A2000000E155801E26FD100018C6B8D6B8A6B13
:103A30008B6BDECF14F0DDCF15F0D890155004E677
:103A4000280E145C000E15584EE2050E7C1901E19B
:103A50007D5101E158D1010E7C5F000E7D5B030EAC
:103A60007C17000E7D177C517D1103E1010E7A6FEA
:103A70007B6B010E7C1905E17D5103E10A0E7A6F23
:103A80007B6B020E7C1905E17D5103E1640E7A6FB8
:103A90007B6B030E7C1904E17D5102E17A697B693D
:103AA000010E7C15146E156A7CC016F07DC017F0EF
:103AB000D89017321632010E1616000E1450161832
:103AC000E8B08180E8A081907CC014F07DC015F042
:103AD000D89015321432010E1414E8B08182E8B087
:103AE00012D1819210D17C517D110FE180B408D0A8
:103AF0006251400B03E08A908A92F8D78A80F6D709
:103B00008A908A92DAEC21F0F9D0010E7C1901E05A
:103B10007AD07D5101E077D080B408D06251400B5B
:103B200003E08A908A92F8D78A80F6D70001E6519E
:103B3000E66E0A0EE66E6BEC24F0E552E552E7C045
:103B400014F0156A1450E66E0B0EE66E6BEC24F062
:103B5000E552E5520F0E0001E815E66E0C0EE66E1A
:103B60006BEC24F0E552E55264C0E6FF080EE66E09
:103B70006BEC24F0E552E5528B6A8A908A92050E2E
:103B800000017C6F7D6B030E9E1935E19F5133E17F
:103B90000001EA51E66E100EE66E6BEC24F0E55281
:103BA000E552EBC014F0156A1450E66E110EE66E85
:103BB0006BEC24F0E552E552ECC0E6FF120EE66E27
:103BC0006BEC24F0E552E55200019651E66E130EBF
:103BD000E66E6BEC24F0E552E55297C014F0156ADE
:103BE0001450E66E140EE66E6BEC24F0E552E552CE
:103BF0005A0EE66E01D0E66A1E0EE66E6BEC24F0FD
:103C0000E552E55280D0020E7C194AE17D5148E12F
:103C10009E519F110FE080B408D06251400B03E029
:103C20008A908A92F8D78A80F6D79E6B9F6B899884
:103C3000899A34D080B408D06251400B03E08A9056
:103C40008A92F8D78A80F6D7905191111BE094514F
:103C500002E1800E951916E0E6C0EAF0E7C0EBF04D
:103C6000E8C0ECF0E9C0EDF094C096F095C097F094
:103C700094C098F095C099F0030E9E6F9F6B898851
:103C8000898A0CD00001EA6BEB6BEC6BED6B0001E9
:103C9000966B800E976F010E9E6F9F6B8A8015D07A
:103CA000030E7C1914E17D5112E180B408D06251F9
:103CB000400B03E08A908A92F8D78A80F6D70001F9
:103CC000E66BE76BE86BE96B8A908A821CD0050E85
:103CD0007C1917E17D5115E180B408D06251400B89
:103CE00003E08A908A92F8D78A80F6D788EC10F0A1
:103CF00000017C6B7D6B010E7A6F7B6B8A908A92E0
:103D000002D080A4FED7060EE15C02E2E16AE55231
:103D1000E16EE552E7CFD9FF1200D9CFE6FFE1CF40
:103D2000D9FF060EE126D950FD0FE96EFF0EDA200D
:103D3000EA6EEE50ED1002E1010E01D0020E00011C
:103D40006C6F6D6BDE6ADD6A7051711119E0B80E2F
:103D50008B1694166451651101E18B8C010E641968
:103D600003E1655101E18B84020E641903E16551A1
:103D700001E18B80030E641903E1655101E18B823F
:103D8000726B736BD950F70FE96EFF0EDA20EA6E93
:103D9000EE50ED1044E1FD0EDBCF14F0FE0EDBCF54
:103DA00015F06851141802E16951151801E187D026
:103DB000010EDE6EDD6A020EDB6A030EDB6A040EA4
:103DC000DB6A050EDB6A78C014F079C015F0166A5C
:103DD000176A15AE02D016681768D950020FE96E3F
:103DE000DACFEAFF1450EE5C1550EE581650EE583C
:103DF0001750EE5864E282AE62D00001685169113A
:103E000002E1F8D901D0FED9D950020FE96EDACF1C
:103E1000EAFFEE2A000EEE22EE22EE22D4D7D9508F
:103E2000F70FE96EFF0EDA20EA6E010EEE1847E199
:103E3000ED5045E1FD0EDBCF14F0FE0EDBCF15F0AB
:103E40006651141802E16751151839E0020EDB6A59
:103E5000030EDB6A040EDB6A050EDB6A78C014F021
:103E600079C015F0166A176A15AE02D01668176881
:103E7000D950020FE96EDACFEAFF1450EE5C15500C
:103E8000EE581650EE581750EE5819E282AE17D081
:103E9000D950FD0FE96EFF0EDA20EA6EEE50ED10FC
:103EA00002E1B0D901D0A6D9D950020FE96EDACF1C
:103EB000EAFFEE2A000EEE22EE22EE22CFD700011C
:103EC000030E7C1910E17D510EE1D950F70FE96E18
:103ED000FF0EDA20EA6E010EEE1805E1ED5003E167
:103EE000010E726F01D0726B736B020EDB6A030EF0
:103EF000DB6A040EDB6A050EDB6AF90EDBCF14F019
:103F0000FA0EDBCF15F0FB0EDBCF16F0FC0EDBCF8D
:103F100017F0D950020FE96EDACFEAFF1450EE5CC9
:103F20001550EE581650EE581750EE5801E3B4D025
:103F300082AEB2D0D950FD0FE96EFF0EDA20EA6EE4
:103F4000EE50ED1016E0E60EE96E000EEA6E00018E
:103F5000EE51EE5CEF51EE58F051EE58F151EE5843
:103F600001E39AD0E62B000EE723E823E92342D9A8
:103F70001AD00001E651E711E811E91106E0E60761
:103F8000000EE75BE85BE95B0DD0D950F70FE96EF7
:103F9000FF0EDA20EA6E010EEE1801E07DD0ED5042
:103FA00001E07AD02FD9FD0EDBCF66F0FE0EDBCF1D
:103FB00067F0D950F70FE96EFF0EDA20EA6EEE5087
:103FC000ED1007E100017451751103E0746B756B1E
:103FD00063D0D950F70FE96EFF0EDA20EA6E010EBA
:103FE000EE1805E1ED5003E1040E801455E0D950C0
:103FF000F70FE96EFF0EDA20EA6E010EEE182FE1E0
:10400000ED502DE10001030E7C1929E17D5127E1DE
:10401000D950FD0FE96EFF0EDA20EA6EEE50ED107A
:1040200007E18D3505E28C510008000E8D5512E335
:10403000D950FD0FE96EFF0EDA20EA6E010EEE1880
:104040000EE1ED500CE18B350AE28A510008000EBA
:104050008B5505E28A6B8B6B8C6B8D6B1DD0F5ECF1
:1040600026F0200E0001B85D03E16D50020B09E05F
:10407000D950F70FE96EFF0EDA20EA6EEE50ED1020
:104080000BE0D950020FE96EDACFEAFFEE2A000EFC
:10409000EE22EE22EE2231D70001725173111DE0A3
:1040A000B80E8B166451651101E18B8C010E6419F9
:1040B00003E1655101E18B84020E641903E165514E
:1040C00001E18B80030E641903E1655101E18B82EC
:1040D00076C0E6FF04EC33F0E5520001726B736BBF
:1040E0009E519F1139E0D950F70FE96EFF0EDA208B
:1040F000EA6E020EEE1801E1ED502EE0020E9E195E
:1041000001E19F5105E0030E9E1926E19F5124E134
:10411000D950FD0FE96EFF0EDA20EA6EEE50ED1079
:104120000EE1F90EDB500001EA5FFA0EDB50EB5BAB
:10413000FB0EDB50EC5BFC0EDB50ED5B0DD0F90EA3
:10414000DB500001EA27FA0EDB50EB23FB0EDB50BD
:10415000EC23FC0EDB50ED23D9CFE9FFDACFEAFFE9
:10416000010EEE1836E1ED5034E1020EDB6A030E6B
:10417000DB6A040EDB6A050EDB6A78C014F079C0D6
:1041800015F0166A176A15AE02D016681768D9506E
:10419000020FE96EDACFEAFF1450EE5C1550EE58CC
:1041A0001650EE581750EE5814E282AE12D00001AD
:1041B0006851691102E126D801D01CD8D950020FEC
:1041C000E96EDACFEAFFEE2A000EEE22EE22EE22B0
:1041D000D4D700017051711101E08B6A6C6B6D6B6B
:1041E000060EE15C02E2E16AE552E16EE552E7CFDC
:1041F000D9FF120000016E516F1102E10AEF21F0A8
:1042000073EF21F000016E516F1102E173EF21F0A5
:104210000AEF21F0030E0001641901E1655141E04C
:10422000020E641901E165512AE0010E641901E1F1
:10423000655114E064514BE1655149E18B8C8B84ED
:104240008B908B9276C0E6FF04EC33F0E5520001D0
:10425000725173113CE18B9C8B8432D08B9C8B848C
:104260008B808B9276C0E6FF04EC33F0E5520001C0
:10427000725173112CE18B9C8B948B8022D08B9C80
:104280008B948B808B8276C0E6FF04EC33F0E55292
:104290000001725173111BE18B9C8B948B908B826C
:1042A00011D08B8C8B948B908B8276C0E6FF04ECC4
:1042B00033F0E55200017251731109E18B8C8B943C
:1042C0008B908B9276C0E6FF04EC33F0E552010E42
:1042D00000016425646F000E6521656F030E64178D
:1042E000000E65171200030E0001641901E165510B
:1042F00041E0020E641901E165512BE0010E6419E1
:1043000001E1655116E064514BE1655149E18B8C47
:104310008B948B908B8276C0E6FF04EC33F0E552F1
:104320000001725173113CE18B9C8B948B908B82BA
:1043300032D08B8C8B848B908B9276C0E6FF04EC12
:1043400033F0E5520001725173112AE18B8C8B948A
:104350000FD08B9C8B848B808B9276C0E6FF04EC15
:1043600033F0E5520001725173111AE18B9C8B847A
:104370008B9010D08B9C8B948B808B8276C0E6FFC9
:1043800004EC33F0E55200017251731109E18B9C8A
:104390008B948B808B9276C0E6FF04EC33F0E55271
:1043A0000001010E645F000E655B030E6417000ED2
:1043B00065171200D9CFE6FFE1CFD9FF0A0EE1263B
:1043C000E6C0DFFF010EE7C0DBFF020EE8C0DBFF47
:1043D000030EE9C0DBFFD9CFE9FFDACFEAFFD880CF
:1043E0003F0EEE54420EEE540F0EEE54000EEE54FD
:1043F00009E23F0EDE6E420EDE6E0F0EDE6EDD6AED
:10440000DD52DD52010EF36E040EF3CFDBFF050E1D
:10441000DB6A080EDB6A090EDB6AD9CFE9FFDACF67
:10442000EAFF0A0EEE5C000EEE58000EEE58000E8B
:10443000EE5807E3020EF36E040EF3CFDBFF050E1A
:10444000DB6AD9CFE9FFDACFEAFF640EEE5C000E3B
:10445000EE58000EEE58000EEE5807E3030EF36E12
:10446000040EF3CFDBFF050EDB6AD9CFE9FFDACF0D
:10447000EAFFE80EEE5C030EEE58000EEE58000E5A
:10448000EE5805E3040EF36EDB6E050EDB6AD9CF42
:10449000E9FFDACFEAFF100EEE5C270EEE58000EB1
:1044A000EE58000EEE5807E3050EF36E040EF3CF40
:1044B000DBFF050EDB6AD9CFE9FFDACFEAFFA00EFA
:1044C000EE5C860EEE58010EEE58000EEE5807E335
:1044D000060EF36E040EF3CFDBFF050EDB6A000160
:1044E0006351010BFCE16351010BFDE0060EDB6A39
:1044F000070EDB6A060EDBCF14F0070EDBCF15F0DC
:10450000040EDBCF16F0050EDBCF17F01550171891
:10451000E8AE02D0173404D01650145C175015586A
:1045200007E2B5D9060EDB2A070EE4E3DB2AE2D761
:1045300080A4FED780B4FED700016351010BFCE1DB
:104540006351010BFDE0D9CFE9FFDACFEAFFA00EFE
:10455000EE5C860EEE58010EEE58000EEE5815E396
:10456000D9CFE9FFDACFEAFFA00EEE5E860EEE5A53
:10457000010EEE5A000EEE5A94D9010EF36E080E9B
:10458000F3CFDBFF090EDB6ADED7D950080FE96EE7
:10459000DACFEAFFEE50ED100BE080A4FED780B436
:1045A000FED700016351010BFCE16351010BFDE0FB
:1045B000D9CFE9FFDACFEAFF100EEE5C270EEE58F6
:1045C000000EEE58000EEE5821E3D9CFE9FFDACF06
:1045D000EAFF100EEE5C270EEE58000EEE58000EAD
:1045E000EE581DE3D9CFE9FFDACFEAFF100EEE5EF9
:1045F000270EEE5A000EEE5AEE5A53D9010EF36E04
:10460000080EF3CFDBFF090EDB6ADFD7D950080FA6
:10461000E96EDACFEAFFEE50ED1001E04CD9D95047
:10462000080FE96EDACFEAFFEE50ED100BE080A440
:10463000FED780B4FED700016351010BFCE163514A
:10464000010BFDE0D9CFE9FFDACFEAFFE80EEE5C1F
:10465000030EEE58000EEE58000EEE5821E3D9CFAF
:10466000E9FFDACFEAFFE80EEE5C030EEE58000E2B
:10467000EE58000EEE581DE3D9CFE9FFDACFEAFF7E
:10468000E80EEE5E030EEE5A000EEE5AEE5A09D90F
:10469000010EF36E080EF3CFDBFF090EDB6ADFD7E6
:1046A000D950080FE96EDACFEAFFEE50ED1001E0C5
:1046B00002D9D950080FE96EDACFEAFFEE50ED10BB
:1046C0000BE080A4FED780B4FED700016351010B3C
:1046D000FCE16351010BFDE0D9CFE9FFDACFEAFF3E
:1046E000640EEE5C000EEE58000EEE58000EEE5812
:1046F00020E3D9CFE9FFDACFEAFF640EEE5C000ECB
:10470000EE58000EEE58000EEE581CE3D9CFE9FF2C
:10471000DACFEAFF640EEE5E000EEE5AEE5AEE5A63
:10472000C0D8010EF36E080EF3CFDBFF090EDB6A73
:10473000E0D7D950080FE96EDACFEAFFEE50ED105E
:1047400001E0B9D8D950080FE96EDACFEAFFEE5090
:10475000ED100BE080A4FED780B4FED700016351BA
:10476000010BFCE16351010BFDE0D9CFE9FFDACF8A
:10477000EAFF0A0EEE5C000EEE58000EEE58000E38
:10478000EE5820E3D9CFE9FFDACFEAFF0A0EEE5C5C
:10479000000EEE58000EEE58000EEE581CE3D9CF76
:1047A000E9FFDACFEAFF0A0EEE5E000EEE5AEE5A8D
:1047B000EE5A77D8010EF36E080EF3CFDBFF090E29
:1047C000DB6AE0D7D950080FE96EDACFEAFFEE5086
:1047D000ED1001E070D8D950080FE96EDACFEAFF8A
:1047E000EE50ED100BE080A4FED780B4FED70001A0
:1047F0006351010BFCE16351010BFDE0D9CFE9FFEF
:10480000DACFEAFFEECF14F0EECF15F0EECF16F0D0
:10481000EFCF17F0145015101610171019E0D9CF5C
:10482000E9FFDACFEAFFD880000EEE54000EEE5416
:10483000000EEE54000EEE540CE2D9CFE9FFDACFB1
:10484000EAFFEE06000EEE5AEE5AEE5A2AD8E7D7E5
:1048500032D800016351010BFCE16351010BFDE013
:104860008A8080A4FED780B4FED78A90000163516D
:10487000010BFCE16351010BFDE00A0EE15C02E279
:10488000E16AE552E16EE552E7CFD9FF120000017F
:104890006351010BFCE18A806351010BFDE08A90BA
:1048A000120000016351010BFCE18A826351010B8C
:1048B000FDE08A92120000016351010BFCE18A8243
:1048C0006351010BFDE06351010BFDE16351010BED
:1048D000FDE08A921200D9CFE6FFE1CFD9FF020EA8
:1048E000E126FE0EDB50A96EFD0EDB50A86EA69EE3
:1048F000A69CA684F250DE6EDD6AF26A550EA76EA3
:10490000AA0EA76EA682DF50F26E0000A1B802D0F8
:104910000000FCD7A694A198020EE15C02E2E16AD5
:10492000E552E16EE552E7CFD9FF1200D9CFE6FF9D
:10493000E1CFD9FFFE0EDB50A96EA69EA69CA680F5
:10494000A850E552E7CFD9FF12006DA205D00001B3
:104950006051611113E01BD00001B8510BE0B805A4
:1049600009E0020EB85D06E0040EB85D03E0100E2B
:10497000B85D06E100016051611109E1898612000C
:10498000200EB85D07E100016051611102E18996D6
:1049900012008986120012001200120012000BEFA2
:1049A00031F012001E0EE66E010EE66EDFEC2DF009
:1049B000E552E552400EE66E300EE66E040EE66EEF
:1049C000E66A010EE66E84EC2EF0146E050EE15ED2
:1049D0001450F3CFB5F0F4CFB6F012006D8400019F
:1049E000080EFE6F070EFF6FFE07000EFF5BFE5105
:1049F000FF11FAE16D941200D9CFE6FFE1CFD9FFA4
:104A0000FD0EDBCF08F0FE0EDBCF09F0720E0818AA
:104A100001E1095033E0E868081802E17F0E091847
:104A20002BE0740E081801E1095024E0750E0818F7
:104A300001E109501DE0730E081801E1095016E06C
:104A4000030E081801E109500FE0020E081801E1F9
:104A5000095008E0010E081801E1095001E010D0EA
:104A6000A1DF0FD09EDF0DD09ADF0BD096DF09D0EB
:104A700092DF07D091DF05D091DF03D0000001D095
:104A800000D0010E00D0E552E7CFD9FF1200D9CFF8
:104A9000E6FFE1CFD9FFE652DF6A04012351030AA2
:104AA0001BE0010A1AE1225118E1DF6ADF50030816
:104AB00014E3DF50EA6A300FE96E040EEA22EF5089
:104AC000E66EDF50EA6A330FE96E040EEA22E55221
:104AD000E750EF6EDF2AEAD72251E552E552E7CFE1
:104AE000D9FF1200D9CFE6FFE1CFD9FF030EE126AF
:104AF000DF6A010EDB6A020EDB6A0001B751740A3D
:104B00004DE0060A01E082D0B551B61102E1000E77
:104B100008D0B5C0E9FFB6C0EAFFEF50800B01E056
:104B2000010E000973E1B5C0E9FFB6C0EAFFEE521D
:104B3000EF50E66ED950010FE96EDACFEAFFE55289
:104B4000E750EE6EED6AD950010FE96EDACFEAFF59
:104B5000000ED880EE54000EED5458E2DF500308EA
:104B60001AE3DF50EA6A300FE96E040EEA22EF50D2
:104B7000E66EDF50EA6A330FE96E040EEA22E55270
:104B8000E750EF6EDF50EA6A300FE96E040EEA225A
:104B9000EF6ADF2AE3D70001740E37D0B351B411A6
:104BA00002E1000E08D0B3C0E9FFB4C0EAFFEF5045
:104BB000800B01E0010E000929E1040EE66E330EC0
:104BC000E66E040EE66E010EE66EE66E84EC2EF0E6
:104BD000146E050EE15E1450F3CFB3F0F4CFB4F0D1
:104BE000400EE66E300EE66E040EE66EE66A010ECC
:104BF000E66E84EC2EF0146E050EE15E1450F3CFD9
:104C0000B5F0F4CFB6F00001720EB76F030EE15CA1
:104C100002E2E16AE552E16EE552E7CFD9FF120008
:104C200004012351030A06E0010A08E1225101E1CF
:104C3000020C000C225101E1030C000C000C0401D9
:104C400023050DE122511AE10001300EC96F040E57
:104C5000CA6F040ECC6FCD6BC10ECB6F1200030E6A
:104C6000235D0CE122510AE10001000EC96F050E1F
:104C7000CA6F040ECC6FCD6BC10ECB6F1200D0DFAC
:104C8000030A15E0010A01E012000401225120E1AB
:104C900026C4D1F027C4D2F00001300ECE6F040E2E
:104CA000CF6F8E0ED36F4A0ED46FD08F12000401D7
:104CB00022510EE126C4D1F027C4D2F00001000E2B
:104CC000CE6F050ECF6F8E0ED36F4A0ED46FD08F7E
:024CD0001200D0
:0E4CD200D9CFE6FFE1CFD9FFE652A09A6A6A79
:104CE000686A706A010EE66EE66AE66A710EE66E42
:104CF0000F0EE66EBDEC32F0146E050EE15E145040
:104D0000160E6F6E9F0E6B6E7B0E696EDF6ADF5044
:104D1000146E156A080E145C000E155810E2DF5070
:104D2000040DF3CFE9FFF4CFEAFF000EE926040EED
:104D3000EA22EE6AEE6AEE6AEE6ADF2AE8D76D8C46
:104D40006E6A6D986D9C68A607D068960001CB6B63
:104D5000D06BD16BD26BF7D70001010EE26FE36F1E
:104D6000E46BE56BD86BDF6A020EDF5C26E2EA6A71
:104D7000DF34FE0BEA36E96EC30EE926000EEA22A6
:104D8000EE6AED6AEA6ADF34FE0BEA36E96EBF0EC0
:104D9000E926000EEA22EE6AED6ADF50EA6ADC0FCD
:104DA000E96E000EEA22EF6ADF50EA6ADE0FE96E72
:104DB000000EEA22EF6ADF2AD7D70001080EC36F80
:104DC000040EC46F160E706E0401200E026F040EE6
:104DD000036F080E016F840E006F0001B96BB86B92
:104DE000E552E552E7CFD9FF1200D9CFE6FFE1CF78
:104DF000D9FFE6520001B80507E16DBA05D0686A2F
:104E000069806988020EB86F6850040B05E069502C
:104E1000040B02E06894BFD86DB250D06850010B0B
:104E200009E06950010B06E054DFA08A0001040E7E
:104E3000B86F68906850100B05E06950100B02E0E5
:104E400095D8689868AC12D069AC0FD0010EE66EA8
:104E5000E66A000EE66EE66A730EE66EE66AFCEC43
:104E600024F0146E060EE15E1450689C6850200B0E
:104E700004E06950200B01E060D86850020B13E099
:104E80006950020B10E0010EE66EE66A000EE66E57
:104E9000E66AE6687F0EE66EFCEC24F0146E060E01
:104EA000E15E14506A6A040E0001E76EB819E8AEBC
:104EB00002D0E73402D0E750B85D02E2A19A38D0C0
:104EC00069A635D0DF6A040EDF5C31E268A62FD018
:104ED0006CCFD9F00001D951780BE842E842E842A2
:104EE000DA6F6896D9B506D0DA51EA6ADE0FE96E54
:104EF000000E05D0DA51EA6ADC0FE96E000EEA22F4
:104F0000EF70DA5102E15ED810D0000EE66EE66A6C
:104F1000D90EE66E000EE66E720EE66EE66AFCECE8
:104F200024F0146E060EE15E1450DF2ACCD7A19A4D
:104F3000E552E552E7CFD9FF120070A015D0BBC0F3
:104F4000E9FFBCC0EAFFEF5080080DE1C3C0E9FFF4
:104F5000C4C0EAFFEF50840806E1BBC0E9FFBCC053
:104F6000EAFF8C0EEF6E7090689A12006984689860
:104F70006D820001010ED86F000EE66EE66AE66EE5
:104F8000E66A750EE66EE66AFCEC24F0146E060E18
:104F9000E15E145012000001D86B000EE66EE66A66
:104FA000E66EE66A740EE66EE66AFCEC24F0146EB9
:104FB000060EE15E14506D92699468A402D0689464
:104FC000FCD71200D9CFE6FFE1CFD9FFE652FD0EA4
:104FD0000001D91553E17E0ED915E8407F0B040D71
:104FE000F3CFBBF0F4CFBCF0000EBB27040EBC2304
:104FF000BBC0BDF0BCC0BEF0BD75BBC0E9FFBCC04E
:10500000EAFFEF503C0BE842E8420D0835E1DF6A69
:10501000080EDF5C23E2BBC0E9FFBCC0EAFF020E62
:10502000E926000EEA22EE50EFCFEAFFE96EEF50DC
:10503000E66EDF50EA6A200FE96E040EEA22E552BE
:10504000E750EF6EBBC0E9FFBCC0EAFF020EE926E5
:10505000000EEA22EE2AEF22DF2ADAD7BBC0E9FFF0
:10506000BCC0EAFF020EE926000EEA22200EEE6E18
:10507000040EED6E0DD807D03AD805D0FD0ED91527
:10508000040801E159D8E552E552E7CFD9FF1200F3
:105090000001C76BE16BE46BE56BDB6BC86BC3C0F6
:1050A000E9FFC4C0EAFFEF9EC375C3C0E9FFC4C0F7
:1050B000EAFFEF9EC375BDC0E9FFBEC0EAFFEF9EE9
:1050C000CB6BCC6BCD6BD06BD16BD26B8CD8000E15
:1050D000E66EE66AE66EE66A030EE66EE66AFCECEB
:1050E00024F0146E060EE15E1450C2EF2BF0020E97
:1050F0000001C85D02E182EF2CF0C86BDB511AE1C0
:10510000BDC0E9FFBEC0EAFFEE52080EEF6EBDC0A3
:10511000E9FFBEC0EAFF020EE926000EEA22200ED9
:10512000EE6E040EED6EBDC0E9FFBEC0EAFF8C0E50
:10513000EF6E1200DB6B1200D9CFE6FFE1CFD9FF93
:10514000E652C3C0E9FFC4C0EAFFEF50400B01E0E4
:10515000010EDF6E0001C375080EB85D08E122C4C0
:105160006EFF6E5002E0100E01D0040EB86FC8053D
:1051700026E1C3C0E9FFC4C0EAFF020EE926000E23
:10518000EA22280EEE6E040EED6E5DDB020E0001CB
:10519000C75D06E1C3C0E9FFC4C0EAFF840E0DD0BD
:1051A000DF5006E1C3C0E9FFC4C0EAFFC80E05D066
:1051B000C3C0E9FFC4C0EAFF880EEF6E0FD0D0AFC6
:1051C0000CD0D351D41107E005D0D4C0FAFF0001B0
:1051D000D351F96EFADF0001D09FC86BE552E5525A
:1051E000E7CFD9FF120004012051600BE842E842EA
:1051F000E842E842E842000901E0120021510C0AAD
:1052000050E00B0A3FE00C0A31E0010A22E00B0AF1
:105210001EE0020A1CE0030A18E0080A10E0010A76
:105220000CE00F0A08E0030A01E012000001CB8F36
:10523000080EB86F12000BEF2BF021EF2DF00001DC
:10524000B90EC96F000ECA6F0CD068EF2BF052EF89
:1052500029F024510001C96FCA6BBA0EC927000E8C
:10526000CA23CB81010ECC6FCB8F12000001CB8FF4
:1052700004012451EA6ABA0FE96E000EEA2222C440
:10528000EFFF1200000EE66EE66AE66EE66A020EB8
:10529000E66EE66AFCEC24F0146E060EE15E145035
:1052A00012001200D9CFE6FFE1CFD9FF030EE126AD
:1052B0000401220510E120511F0B00090CE100013F
:1052C000CB8F030E0401215D04E10001010ED76FB5
:1052D00002D00001D76B0401225101E003D120511B
:1052E0001F0B020801E0FED024510F0B000901E161
:1052F000F9D024510F0B010801E2F4D0200E000177
:10530000B85D01E0EFD0CB8F040124BF16D024514B
:105310000F0BE96EEA6AD890E936EA36BF0EE92645
:10532000000EEA22EECFDEFFEDCFDDFF24510F0BA2
:10533000EA6ADE0FE96E000E15D024510F0BE96EFC
:10534000EA6AD890E936EA36C30EE926000EEA2268
:10535000EECFDEFFEDCFDDFF24510F0BEA6ADC0F4D
:10536000E96E000EEA22020EEFCFDBFFD950020FEA
:10537000E96EDACFEAFFEF50010B03E1000EDF9494
:1053800001D0DF8424BF0BD024510F0BE96EEA6AF1
:10539000D890E936EA36BF0EE926000E0AD024512D
:1053A0000F0BE96EEA6AD890E936EA36C30EE926B1
:1053B000000EEA22DECFEEFFDDCFEDFF030E215D12
:1053C00020E1DECFE9FFDDCFEAFFEF50800B11E0F7
:1053D00024BF07D024510F0BEA6ADE0FE96E000EDE
:1053E00006D024510F0BEA6ADC0FE96E000EEA22A8
:1053F000EF82840EDECFE9FFDDCFEAFFE850EF1247
:1054000071D0DF74DECFE9FFDDCFEAFFEF50800B14
:105410001BE0DECFE9FFDDCFEAFFEF9EDECFE9FF45
:10542000DDCFEAFFEF8C020EE66EE66ADECFE6FF26
:10543000DDCFE6FF050EE66EE66AFCEC24F0146EA6
:10544000060EE15E145005D0DECFE9FFDDCFEAFFA6
:10545000EF8CDF74D950020FE96EDACFEAFFEF501C
:10546000020B0EE1DECFE9FFDDCFEAFFEF50800B4C
:1054700032E0DECFE9FFDDCFEAFFEF50040B2BE196
:10548000040124BF07D024510F0BEA6ADE0FE96E36
:10549000000E06D024510F0BEA6ADC0FE96E000EF5
:1054A000EA22EF923B0E146EDECFE9FFDDCFEAFF7A
:1054B000E850EF16020EE66EE66ADECFE6FFDDCFBD
:1054C000E6FF050EE66EE66AFCEC24F0146E060EAE
:1054D000E15E145007D03B0EDECFE9FFDDCFEAFFDF
:1054E000E850EF16030EE15C02E2E16AE552E16E7C
:1054F000E552E7CFD9FF12000001E2514DE1010E64
:10550000E26FE35149E1010EE36F020EC85D0DE168
:10551000C3C0E9FFC4C0EAFFEE52EF6AC3C0E9FFAF
:10552000C4C0EAFFC80EEF6E1200C80535E1DB6BA0
:10553000BBC0E9FFBCC0EAFFEE52080EEF6EBBC075
:10554000E9FFBCC0EAFF020EE926000EEA22200EA7
:10555000EE6E040EED6EBBC0E9FFBCC0EAFF840E28
:10556000EF6E010EDB6FBDC0E9FFBEC0EAFFEE5279
:10557000080EEF6EBDC0E9FFBEC0EAFF020EE926CD
:10558000000EEA22200EEE6E040EED6EBDC0E9FFA5
:10559000BEC0EAFF800EEF6E12000001E46BE56B07
:1055A000020EC85D18E1BDC0E9FFBEC0EAFFEE52C1
:1055B000080EEF6EBDC0E9FFBEC0EAFF020EE9268D
:1055C000000EEA22280EEE6E040EED6EBDC0E9FF5D
:1055D000BEC0EAFF1DD0CC510401265D0001CD51B3
:1055E0000401275904E226C4CCF027C4CDF02BD9FE
:1055F000C3C0E9FFC4C0EAFF020EE926000EEA229A
:10560000280EEE6E040EED6EC3C0E9FFC4C0EAFFC3
:10561000C80EEF6E1200800E0401205D58E10001FB
:10562000C00ECB6F04012351030A2FE0010A09E0E9
:10563000030A4BE10001E60EC96F620ECA6F120E3B
:105640003ED02251F66EF76AD890F636F736960EAF
:10565000F626630EF7220900F5CFC9F00A00F5CF50
:10566000CAF0020E0001F76AC925F66ECA51F72288
:105670000800F5CFCCF0030EF76AC925F66ECA51C3
:10568000F7220800F5CFCDF01200030E225D1AE2DA
:105690002251F66EF76AD890F636F736980EF6264F
:1056A000630EF7220900F5CFC9F00A00F5CFCAF062
:1056B000C9C0F6FFCAC0F7FF0800F5500001CC6F63
:1056C000CD6B12000001CB6B12000001CB6B1200FE
:1056D000D9CFE6FFE1CFD9FF020EE1260401286B06
:1056E000296B20511F0B020A11E0030A0CE0010A8A
:1056F00035E10001CB8F040128810001D7052EE19F
:10570000040128832BD00001CB8F28D00001CB8F40
:10571000040124BF0BD024510F0BE96EEA6AD89024
:10572000E936EA36BF0EE926000E0AD024510F0BE7
:10573000E96EEA6AD890E936EA36C30EE926000E29
:10574000EA22EECFDEFFEDCFDDFFDECFE9FFDDCFDA
:10575000EAFFEF50040B02E0010E286F0001CBAF0F
:1057600007D0280EC96F040ECA6FCB81020ECC6F12
:10577000020EE15C02E2E16AE552E16EE552E7CF3A
:10578000D9FF12006D980001CBBF2BD0D0AF09D04C
:10579000020EC86FE55101E100DF0001E36BE26B2F
:1057A0001200BDC0E9FFBEC0EAFFEE52080EEF6E68
:1057B000BDC0E9FFBEC0EAFF020EE926000EEA22E4
:1057C000200EEE6E040EED6EBDC0E9FFBEC0EAFF16
:1057D0008C0EEF6EC3C0E9FFC4C0EAFF840EEF6E0B
:1057E0001200040120AF0DD00001010EC86FE4517A
:1057F00001E1D3DE0001E36BE26BE15123E17CEFD9
:105800002AF00001020EC86FBDC0E9FFBEC0EAFF6A
:10581000EE52080EEF6EBDC0E9FFBEC0EAFF020EF9
:10582000E926000EEA22200EEE6E040EED6EBDC0DB
:10583000E9FFBEC0EAFF840EEF6EE36BE26BE1515D
:1058400001E15ADE1200D9CFE6FFE1CFD9FFE652DF
:10585000080EDF6E0001CC5D000ECD590AE2CCC00F
:10586000DFFFC75102E1010E03D0C70502E1020EBE
:10587000C76FDF50156AE850CC5DCC6F1550CD591D
:10588000CD6FC3C0E9FFC4C0EAFFEE52DFCFEFFF28
:10589000280ED56F040ED66FCBB118D0DF502DE097
:1058A000C9C0F6FFCAC0F7FFC92B000ECA23080003
:1058B000F550E66ED5C0E9FFD6C0EAFFD52B000E45
:1058C000D623E552E750EF6EDF06E8D7DF5015E04C
:1058D000C9C0E9FFCAC0EAFFC92B000ECA23EF50B6
:1058E000E66ED5C0E9FFD6C0EAFFD52B000ED62361
:1058F000E552E750EF6EDF06E9D7E552E552E7CF14
:10590000D9FF1200D9CFE6FFE1CFD9FF020EE12681
:10591000BBC0E9FFBCC0EAFFEE52EFCFDFFFDFCF35
:1059200014F014500001D15D000ED25902E2D1C032
:10593000DFFFDF50146E156AE850D15DD16F15504E
:10594000D259D26F010EDB6ADF50F36E010EDBCF4E
:10595000F4FFF350F45C16E2010EDB50EA6A280F04
:10596000E96E040EEA22EF50E66ECEC0E9FFCFC02A
:10597000EAFFCE2B000ECF23E552E750EF6E010E6B
:10598000DB2AE2D7000ED880D155000ED25527E28F
:10599000BDC0E9FFBEC0EAFFEE52080EEF6EBDC00B
:1059A000E9FFBEC0EAFF020EE926000EEA22280E39
:1059B000EE6E040EED6EBBC0E9FFBCC0EAFFEF5017
:1059C000400B06E1BDC0E9FFBEC0EAFFC80E05D02E
:1059D000BDC0E9FFBEC0EAFF880EEF6E28D0BDC093
:1059E000E9FFBEC0EAFFEE52080EEF6EBDC0E9FF50
:1059F000BEC0EAFF020EE926000EEA22200EEE6E7D
:105A0000040EED6EBDC0E9FFBEC0EAFF840EEF6E6E
:105A1000D351D41107E005D0D4C0FAFF0001D3510F
:105A2000F96EFADF0001D09FE15101E165DD020E60
:105A3000E15C02E2E16AE552E16EE552E7CFD9FFAF
:105A40001200D9CFE6FFE1CFD9FFE6520001CB8F9C
:105A5000010EE66EE66AE66A710EE66E0F0EE66EFF
:105A6000BDEC32F0146E050EE15E1450DF6ADF50BB
:105A7000146E156A080E145C000E155810E2DF5003
:105A8000040DF3CFE9FFF4CFEAFF000EE926040E80
:105A9000EA22EE6AEE6AEE6AEE6ADF2AE8D76D8CD9
:105AA000010EE66EE66AE66ABA0EE66E000EE66E75
:105AB000BDEC32F0146E050EE15E14506D9C0001D9
:105AC000080EC36F040EC46F000EBB6F040EBC6FD4
:105AD000BBC0BDF0BE6F22C4B9F0B95102E1100ED7
:105AE00012D0010EE66EE66AB90EE66E000EE66EA4
:105AF000010EE66EE66AFCEC24F0146E060EE15E22
:105B000014500001200EB86FE552E552E7CFD9FFDF
:105B10001200D9CFE6FFE1CFD9FF020EE126000E39
:105B2000DE6E040EDD6EFD0EDB50E824166EFE0EFA
:105B3000DB50040DF3501624040DF4CF15F0D9CF2B
:105B4000E9FFDACFEAFFF350EE261550ED22DECF63
:105B5000E9FFDDCFEAFFEF9EFD0EDB500AE1FE0E0E
:105B6000EA6ADB34FE0BEA36E96EBF0EE926000E68
:105B700009D0FE0EEA6ADB34FE0BEA36E96EC30E8C
:105B8000E926000EEA22DECFEEFFDDCFEDFFDECF0D
:105B9000E9FFDDCFEAFFEF9CDECFE9FFDDCFEAFFD3
:105BA000040EE926000EEA22EF8C020EE15C02E20E
:105BB000E16AE552E16EE552E7CFD9FF1200D9CF95
:105BC000E6FFE1CFD9FF020EE126FD0EDBA407D0F0
:105BD000E66AFE0EDBCFE6FF9CDFE552E552FD0EE6
:105BE000DBA208D0010EE66EFE0EDBCFE6FF91DFF2
:105BF000E552E552FE0EDB50156A700F146E0F0E63
:105C0000152214C0DEFF15C0DDFFDECFE9FFDDCFBA
:105C1000EAFFFD0EDBCFEFFF020EE15C02E2E16A7C
:105C2000E552E16EE552E7CFD9FF1200D9CFE6FF8A
:105C3000E1CFD9FF020EE126FE0EDB5020E1BDC010
:105C4000E9FFBEC0EAFFEE52080EEF6EBDC0E9FFED
:105C5000BEC0EAFF020EE926000EEA22200EEE6E1A
:105C6000040EED6EBDC0E9FFBEC0EAFF8C0EEF6E04
:105C7000C3C0E9FFC4C0EAFF840EEF6E3BD0FD0E47
:105C8000DB50E824166EFE0EDB50040DF350162494
:105C9000040DF3CF14F0F4CF15F0000E1426040E0B
:105CA000152214C0DEFF15C0DDFF840EDECFE9FF34
:105CB000DDCFEAFFE850EF12FD0EDB50E824166E50
:105CC000FE0EDB50040DF3501624010F040DF3CF2C
:105CD00014F0F4CF15F0000E1426040E152214C093
:105CE000DEFF15C0DDFF840EDECFE9FFDDCFEAFF6A
:105CF000E850EF12020EE15C02E2E16AE552E16E69
:105D0000E552E7CFD9FF1200D9CFE6FFE1CFD9FFA7
:105D1000020EE126FD0EDB500AE0FE0EEA6ADB34DD
:105D2000FE0BEA36E96EC30EE926000E09D0FE0E20
:105D3000EA6ADB34FE0BEA36E96EBF0EE926000E96
:105D4000EA22EECFDEFFEDCFDDFFD9CFE9FFDACFDC
:105D5000EAFFEE50ED1003E1F36AF46A44D0DECFBF
:105D6000E9FFDDCFEAFF020EE926000EEA22FB0E74
:105D7000DBCFEEFFFC0EDBCFEDFFDECFE9FFDDCFAB
:105D8000EAFFEE52FA0EDBCFEFFF400EDECFE9FF67
:105D9000DDCFEAFFE850EF16880EDECFE9FFDDCF5A
:105DA000EAFFE850EF12FD0EDB500AE0FE0EEA6A51
:105DB000DB34FE0BEA36E96EC30EE926000E09D08D
:105DC000FE0EEA6ADB34FE0BEA36E96EBF0EE92608
:105DD000000EEA22EF74DECF14F0DDCF15F014C010
:105DE000F3FF15C0F4FF020EE15C02E2E16AE55246
:105DF000E16EE552E7CFD9FF1200D9CFE6FFE1CF40
:105E0000D9FF6DA84ED0FE0EEA6ADB34FE0BEA36EF
:105E1000E96EC30EE926000EEA22EE50EFCFEAFF4C
:105E2000E96E400EEE16EE6AEE6AEE6AFE0EEA6A61
:105E3000DB34FE0BEA36E96EC30EE926000EEA22D9
:105E4000EE50EFCFEAFFE96EEE7CFE0EEA6ADB343D
:105E5000FE0BEA36E96EC30EE926000EEA22EF7465
:105E6000400E146EFE0EEA6ADB34FE0BEA36E96E73
:105E7000C30EE926000EEA22EE50EFCFEAFFE96EEC
:105E80001450EF16FE0EEA6ADB34FE0BEA36E96EBA
:105E9000C30EE926000EEA22EE50EFCFEAFFE96ECC
:105EA000EF7CE552E7CFD9FF12006D6A696A000105
:105EB000B86B12000001B85115E180A213D06D6AD1
:105EC000696A160E6F6E9F0E6B6E7B0E696ED08EBA
:105ED000A28AA08AF28E6DB602D06D86FCD7000130
:065EE000010EB86F120074
:0A5EE600019E08D0019E09AE05D010
:105EF000086C091EE86A0922018E09C003F008C077
:105F000002F0136A126A8E0E046E056AA1EF30F079
:105F1000016ADDEC30F0F5EC30F001B685EF30F0E1
:105F200001A205D001B885EF30F08CEF30F001AA66
:105F300005D001B085EF30F08CEF30F001B002D029
:105F400001A802D098EF30F0056A0F500A24046EC1
:105F5000E86A05227E0E045EE86A055A126A136A30
:105F6000026A036A0E500902F4CF03F0F3CF02F085
:105F70000D500902F3501326F4500222000E0322A2
:105F80000E500802F3501326F4500222000E032292
:105F90000C500902F3501226F4501322000E022274
:105FA00003220D500802F3501226F4501322000E63
:105FB000022203220E500702F3501226F45013223D
:105FC000000E022203220C500802F4501226000E8A
:105FD0001322022203220D500702F4501226000E53
:105FE000132202220322A1EF30F0006AE86A0EAE0B
:105FF00002EF30F00B6C0C1E0D1E0E1E0C220D223B
:106000000E22001E09AE0DEF30F0066C071E081EB2
:10601000091E072208220922001E99EC32F009BE4F
:1060200024EF30F000AE000C066C071E081E091E9F
:10603000E86A072208220922026C031E041E051EBC
:10604000032204220522000C00BE14EF30F0018868
:10605000FF0C09C013F008C012F008500D02F4CF75
:1060600007F0F3CF06F009500E02F4CF09F0F3CF9A
:1060700008F00D02F3500726F4500822E86A0922BE
:1060800012500E02F3500726F4500822E86A092243
:106090000EAE4FEF30F01250085E1350095A13AE97
:1060A000000C0D50085E0E50095A000C016ADDEC20
:1060B00030F001B660EF30F001A20ED001B405D08F
:1060C0007F0E096EFF0E086E1FD0800E096E086AE3
:1060D0001BD0096A086A18D001B0FBD78F0E0A607E
:1060E000EDD77E0E0A64F5D78E0E0A5C05E0D890D7
:1060F000093208320A2AF8D701A406D0086C091E12
:10610000E86A092209AEE5D712007F0E0A6EFF0E7B
:10611000096E086E076E12007F0E01BEFF0E0A6E3A
:1061200002D07F0E0A6E800E096E086A076AF3D7E6
:1061300001AE04D0800E0A6E096AF7D70A6A096AAE
:10614000F4D70350021013101210F8E005BEF0D778
:1061500003BE0CD004500510EBE0D8901236133675
:10616000023603360406D8A00506F2D70550D4E15E
:106170000428D2E012AE11D07F0E121402E113A057
:106180000CD0132AE86A0222032207E3D8800332E4
:1061900002321332042A0428BFE00450C9E013C0BD
:1061A00007F002C008F00334096E04300A6E0932A9
:1061B0000A9E01BE0A8E8BEF30F009360A3602E3E2
:1061C0000184017E06E101800A6A096A086A076A99
:1061D00012000A2803E0D88009321200D890093250
:1061E00002E101821200018612000E360F3602E330
:1061F000018C017E06E101880F6A0E6A0D6A0C6A45
:1062000012000F2803E0D8800E321200D8900E3210
:06621000EAE1018A120020
:0A621600040120511F0B010801E0F4
:106220001200245101E01200060E215D1EE12351EF
:10623000230A1BE0010A0CE0030A17E10001B9057B
:1062400014E100010A0EC96F630ECA6F090E09D06E
:106250000001B9050AE10001670EC96F630ECA6F3C
:106260002F0ECC6FCD6BC00ECB6F04012051600B95
:10627000E842E842E842E842E842010801E0120050
:1062800021510B0A2AE0080A1DE0090A15E0080A54
:1062900009E00B0A05E0080A01E012001FEF26F0F2
:1062A0003FEF26F00001400EC96F040ECA6F010EC9
:1062B000CC6FCD6BC10E0FD00001800ECB6F23C40D
:1062C00040F412000001410EC96F040ECA6F010EA6
:1062D000CC6FCD6B810ECB6F12000001800ECB6FA7
:0662E00022C441F412008B
:0A62E6001201000200000008D804B5
:1062F00012F801000102000109022900010100C099
:10630000320904000002030000000921110100010C
:10631000222F00070581034000010705010340000B
:1063200001040309042A034D006900630072006F31
:10633000006300680069007000200054006500637D
:106340000068006E006F006C006F00670079001835
:1063500003470065006E006500720069006300205D
:106360000048004900440006A0FF0901A1010903FB
:10637000150026FF00750895048102090415002602
:10638000FF007508950491020905150026FF0075A8
:0E639000089504B102C0F862216325634F63D3
:02639E001E0ED1
:1063A000F66E100EF76E000EF86E04010900F5503F
:1063B0003B6F0900F5503C6F03E13B6701D03DD0D6
:1063C0000900F550366F0900F550376F0900F55098
:1063D000386F09000900F550E96E0900F550EA6EC2
:1063E000090009000900F550396F0900F5503A6FAE
:1063F00009000900F6CF3DF4F7CF3EF4F8CF3FF4A3
:1064000036C4F6FF37C4F7FF38C4F8FF0401395328
:1064100002E13A5307E00900F550EE6E3907F8E261
:106420003A07F9D73DC4F6FF3EC4F7FF3FC4F8FF73
:0C64300004013B07000E3C5BBFD71200CC
:04643C00FF0EE36606
:1064400024EF32F040EF32F0FE0EE3662AEF32F036
:106450002CEF32F0FF0EE32AFE0EE3060CE0E3061B
:106460000AE0E30608E00000000000000000000071
:10647000FE0EE306F9E1FF0EE306F6E150EF32F01F
:10648000FE0EE3060DE0E3060BE0E30609E0000084
:1064900000000000000000000000FE0EE306F9E12D
:1064A0001200000EF36E00EE00F0080E01D812008C
:1064B000EA6002D0EE6AFCD7F350E9601200EE6A9F
:0264C000FCD707
:0E64C20006500B02F3CF02F0F4CF03F00C02F1
:1064D000F3500326000EF420046E06500D02F35014
:1064E0000426000EF420056E06500E02F350052619
:1064F00007500B02F3500326F4500422000E05222D
:1065000007500C02F3500426F450052207500D02E8
:10651000F350052608500B02F3500426F4500522D0
:1065200008500C02F350052609500B02F3500526C3
:02653000120057
:0E653200056A046A036A026A200EE76ED890BA
:10654000063607360836093602360336043605366F
:106550000B50025C0C5003580D5004580E50055857
:1065600009E30B50025E0C50035A0D50045A0E50B2
:0A657000055A062AE72EE4D71200B0
:06657A00FE0EE3CFE9FF75
:10658000FF0EE3CFEAFFE9CFF3FFEACFF4FFFB0E04
:10659000E35003E1FC0EE35009E0FB0EE30602E2E8
:0E65A000FC0EE306FD0EE350EE6EF1D7120086
:0265AE00FF0EDE
:1065B000E3501D6EEF0E01D0F30EE76EE72EDEEF17
:1065C00032F00C0E1C6EE76AE72EE4EF32F01C2E60
:0C65D000E3EF32F01D2EDCEF32F0120081
:0465DC00056A046ADE
:1065E000100EE76ED89008360936043605360D5081
:1065F000045C0E50055805E30D50045E0E50055A1C
:08660000082AE72EF0D7120072
:08660800FF0EE3501D6E480E69
:1066100001D04C0EE76EE72EFED7E76AE72EFED7D5
:086620001D2EF7D70000120047
:0866280013EE00F023EE00F078
:10663000F86A019CCFEC31F003EC08F0F4EC0BF0BD
:04664000FBD7120072
:0C664400FF0EE3501D6E1B0E00D001D0B5
:10665000200EE76EE72EFED71D2EFAD700D01200CF
:106660000100000000000000000000000000000029
:1066700000000000000028000100010000000000F0
:10668000000000000000000000000000000000000A
:1066900000000000000000000000000000000000FA
:1066A00000000000000000000000000000000000EA
:0866B00000000100000000726F
:020000040030CA
:0100000028D7
:010001000EF0
:010002003FBE
:010003001EDE
:010005008179
:010006008178
:010008000FE8
:01000900C036
:01000A000FE6
:01000B00E014
:01000C000FE4
:01000D0040B2
:00000001FF
